:030000000219FDE5
:03000B000200AA46
:03002B000201656A
:03005B000202FBA3
:030073000202E1A5
:1000800002030406080C10182030406080040608A3
:100090000C10182030406080A0C000070F1F3F0DDB
:1000A0000D0403060D0503030202C2AFC0D0C0E079
:1000B000206217E5256002E473E525F4F58A758B67
:1000C00000D262D0E0D0D0D2AF3285268AC262E5BB
:1000D00026F46035306803207210758B00D0E0D0B4
:1000E000D0D295D293D297D2AF32D295D293D29723
:1000F000206E0C2066097406D5E0FDE57E42907501
:100100008B00D0E0D0D0D2AF32758A00C28DD262DF
:1001100001FF01B9306805206602C29501B9306857
:1001200005206602C29701B9306805206602C293B5
:1001300001B9C29430680A2066077406D5E0FDC292
:100140009501B9C29630680A2066077406D5E0FDAD
:10015000C29701B9C29230680A2066077406D5E0DA
:10016000FDC29301B9C2AFC2AD53E6EFC0D0C0E04B
:10017000D2D3D2AFC2CEE52A6007207449152A2116
:10018000C67800790020742EE580307E01F430E5D9
:100190000278FF53DACF207E0343DA20307E034318
:1001A000DA10C2D8C271E580307E01F430E5027900
:1001B000FFC3E89970CB306103752A402074037542
:1001C0002A40885FD27020740DE52B6004152B2126
:1001D000D643DA01C2D820700221E9A85F2061026B
:1001E000C27020740221E788227882B60403852237
:1001F00024C3E52594404002D26420CF0AD0E0D049
:10020000D043E610D2AD32C2CF053A7802E52A607B
:1002100005307402152AC3E55F940140057562003C
:100220004133756300756C00E5622401F56250038B
:100230007562FF7982B7020D306D1DC3E5229432DD
:100240004016854D227982B7030E306D0BC3E5222F
:1002500094324004798E8722C3E5239522600840BA
:1002600004152341670523D8CA056CE56C70021597
:100270006CD56D63756D017805C3E56C956E40575F
:10028000C3E56C956F50087801756D0302029BC33E
:10029000E56C957050057801756D01C3E565952491
:1002A000401E7982B7040241CC206D14852465E597
:1002B0006C046003856E6C756D0175233C0202D77A
:1002C000E5652850057565FF41CCF565E565047069
:1002D000067563FF756CFFD0E0D0D043E610D2AD59
:1002E00032C2AFC0D053E67FC2607591008556948C
:1002F000855795759104D0D0D2AF32C2AF53E6EF97
:10030000C2ADC0D0C0E0C0F0D2D3D2AFA8FBA9FC30
:10031000C2D8307102616253DACF207E0343DA1013
:10032000307E0343DA20D271E580307E01F420E58F
:1003300002613988278928A14753DACF207E0343F9
:10034000DA20307E0343DA10C2D8C271307402A1C1
:10035000337800E580307E01F430E502A133885F18
:10036000A11B53DACF207E0343DA20307E0343DA29
:1003700010C271206102813B53DACF207E0343DA41
:1003800010307E0343DA20C2D8D271885A895BC309
:10039000E89558F8E99559F97B007E087A00C3E89A
:1003A000948CE994005005755E00812D882178A217
:1003B000E6A8216055C3E894C8E994005008E4D247
:1003C000E4FB7A0A8108C3E89468E994015008E4E0
:1003D000D2E3FB7A0F8108C3E894D0E99402500875
:1003E000E4D2E2FB7A1E8108C3E894A0E9940550A8
:1003F00008E4D2E1FB7A3C8108C3E89498E99408C8
:100400005008E4D2E0FB7A787E00C3E8955CFCE912
:10041000955DFD30E70AECF42401FCEDF43400FDB9
:10042000755E00C3EC9AED9E5003755E01885C8991
:100430005D855A58855B597802A11BC3E89527F85A
:10044000E99528F9307C0281FF307B0281FF307A08
:100450000281F8207502815EE9FDE8FC817DE9C337
:1004600013F9E813F830790281F8E9C313F9E813B6
:0D047000F830780281F8E9C313FDE813FCB1
:10047D0020612CC3EC941CED940240028194ED702C
:10048D001EC3EC94C850180529E52970021529C31F
:10049D00E529940A5002A133755F00D270A133E5AE
:1004AD0029600215297400207F037896E624FAFE50
:1004BD00E43400FFC3EC9EFCED9FFD5006780079FF
:1004CD000081FFC3EC94FFED9400400678FF7900A6
:1004DD0081FFEC8575F0A4C5F0A2F733F8790040E3
:1004ED000302051B78FF790002051BE9C313F9E828
:1004FD0013F8307C0EE9600278FFC3E81338F8E496
:10050D003400F9C3E894FFE99400400278FF885F56
:10051D00D270206102A133741FF4552F4BF52FC2F9
:10052D0074EB7002D274752A40307403752A0A3048
:10053D006102A14720740353DAFE207403752B204A
:10054D00D0F0D0E0D0D0D2AD43E610327901020523
:10055D00777903020577790A020577791E02057707
:10056D00796402057779C80205777817E4D5E0FD3F
:10057D00D8FAD9F6227A147B7802059E7A107B8CF4
:10058D0002059E7A0D7BB402059E7A0B7BC802058F
:10059D009E7902B27DE4C296D5E0FDC297D5E0FD0D
:1005AD00D297D5E0FDD296D5E0FDC295E576D5E0A2
:1005BD00FDD2957496D5E0FDD9D9EAF8D5E0FDD8F0
:1005CD00FBDBCEC29622C37C007D0075F00005F0EA
:1005DD00EA33FAEB33FB50F6EB13FBEA13FAC3E9FC
:1005ED00FFE8FEE89AF8E99BF95004EFF9EEF8B34D
:1005FD00EC33FCED33FDD5F0DFEDF9ECF822E889B5
:10060D00F08A20D2D4F8A9F07B0030F70B7BFFF4F1
:10061D002401F8E9F43400F9E88520F0A4ADF0F8F0
:10062D00E98520F0A4AFF0FEED2EF974003FFA7CC1
:10063D0004C3EA13FAE913F9E813F8DCF48BF0308C
:10064D00F70AE8F42401F8E9F43400F9E889F0C276
:10065D00D4F8A9F0227882B60403020701C3E55F3E
:10066D009419401EE52D54067018206D36780579C5
:10067D0094E7146007780A1460027812C3E5419874
:10068D00401F306D09856765756CFF756D0185229D
:10069D0024E4F545F546F547F548F549C26D0207E1
:1006AD0001D26D7994E7147013E523F43333F91304
:1006BD00F8E9540104F9E854FE0206F5E714147044
:1006CD0014E523F4333333F913F8E9540304F9E84B
:1006DD0054FC0206FDE523F433333333F913F8E903
:1006ED0054070404F9E854F8C39440F8E99400F968
:1006FD008845894622C3E54113F9E54013F8C3E562
:10070D004598F8E54699F9500CC3E89480E994FFB3
:10071D004016020739C3E8947FE99400500302079D
:10072D0039787F7900020739788079FF884A894BBB
:10073D0022E54A2547F8E54B3548F9854B20E4304D
:10074D000701F43549FA30E709C3EA94F040150280
:10075D000777C3EA940F500302077778FF79FF7A82
:10076D000F020777780079007AF0C3E5249564507D
:10077D000AC374019524500B020795E54B20E70E33
:10078D00020795E54B30E706884789488A49227864
:10079D00A4E6FAC3E54A33F8E54B33F9D10BE9305A
:1007AD00E70BC3E89480E994FF4013E1CFC3E894CD
:1007BD007FE994005002E1CF787F7900E1CF788016
:1007CD0079FFE820E715C3E52398F84009C3E894BD
:1007DD000140030207F678010207F6E8F42401252B
:1007ED0023F840030207F678FF884C2278A5E6FA35
:1007FD00A848A94912060BE930E70CC3E89401E9B2
:10080D0094FF401602082BC3E894FFE994005003AF
:10081D0002082B78FF790002082B780179FFE92077
:10082D00E715C3E54C98F84009C3E894014003026D
:10083D0008527801020852E8F42401254CF84003CF
:10084D0002085278FF88242278FFC26420693D2077
:10085D006A12D264C3E541940A4009C3E525944068
:0F086D005002C26479A1E76023E541601F74FF68
:10087C008541F0848539F0306A0375F005A4F8C51C
:10088C00F0600278FFC3E895675002A8678866227B
:10089C00C3E5409440E5419401E56650031401AD75
:1008AC00046002F566227883E6F520120F4B75E89A
:1008BC009012055975E890E5E820ECFBA8BDA9BE9F
:1008CC00120FE5757155757200C3740013FD7455E4
:1008DC00606613FC74552CFC74003DFDECFAEDFBCA
:1008EC00C3E89AE99B4014E5712455F571E572341F
:1008FC0000F572EA2CFAEB3DFB80E5AE71AF72C3EA
:10090C00E57213F9E57113F8C3E913F9E813F87AF2
:10091C0003C3E913F9E813F8DAF7AA201A7009757A
:10092C0071007572000209441AEA6008EE28FEEFA5
:10093C0039FFDAF88E718F722275E890227883E68F
:10094C00FFE5E820ECF7A8BDA9BE0573C3E57394D9
:10095C00084052757300E9FA79A0E76044EA700721
:10096C00E574601B02097FC3E895746010E5745050
:10097C0006600C1402098B0460F902098BE574F50E
:10098C0074C3946D401B7564C0C3940440137564A8
:10099C0080C39404400B756440C394044003756495
:1009AC000075BB0822EFC39401601F7455601BC314
:1009BC00E894FFE994035012C3E89571E9957250DD
:1009CC0009E564600C15640209DDE564F460020558
:1009DC0064A864C3E524985002A824C3E895654034
:1009EC000AA865E565F4600385656488258826E5B5
:1009FC0073B4070375BB1022743279A687F0A4C5B3
:100A0C00F0A2F733F8C3E895644002A86488228802
:100A1C0024882588268867227540007541F022C2FB
:100A2C00AF75C820A8CCA9CDAA3A30CF010A75C899
:100A3C0024D2AFAB3BAC3C883B893CC3E89BF8E988
:100A4C009C206908F93067026140419DAD3D8A3DAB
:100A5C00F9EA9DFA600478FF79FFAE3EAF3F8B3E1A
:100A6C008C3FC3EC9FFCC3E99CF542A83BA93CC35B
:100A7C00E89EF8E99FF9C3E54113FBE54013FAE85A
:100A8C002AF540E93BF54150067540FF7541FF41A1
:100A9C00E7AA40AB41AC40AD417E047F02C3EB946E
:100AAC000440021E1FC3EB940840021E1FC3ED132B
:100ABC00FDEC13FCDEF7C3EA9CFAEB9DFBEF60093F
:100ACC00C3E913F9E813F8DFF7EA28FAEB39FB8AE4
:100ADC00408B4150067BFF8B408B41C3EB94025003
:100AEC0002D2673069047F0361127892E6FFC3E596
:100AFC0037948240110FC3E53794A040010FC3EF28
:100B0C00940640027F057E05E541C4540FF9E5418A
:100B1C00C454F0F8E540C4540F28F8C3E89EFAE931
:100B2C009400FB4009C3EA9402EB940050047A024F
:100B3C00E4FB618CAA40AB41EBC4FEEAC4540F4EFB
:100B4C00FCC3EA9CFAEB9400FBC3E813C313F8EA6A
:100B5C0028FAEB3400FB8A408B41C3EB9402400231
:100B6C00C2677805EBC4FE7B00EAC4540F4EFAC38F
:100B7C00EA98FA4005C3940250027A027892E6FF92
:100B8C00306002618C855256855357D26043E680A3
:100B9C00C3E49AF8E49BF93067028126E8FAE9FB92
:100BAC00D3E913FDE813FC88528953C3EF94036017
:100BBC0038EF20E00DE82CF8E93DF9ECFAEDFB02FA
:100BCC000BE1E828F8E939F9C3E82402F8E9340024
:100BDC00F97AFE7BFFC3EF9403400E8A548B558841
:100BEC004E894F8C508D51815A885489558A4E8B21
:100BFC004F8C508D51306920C3E53394034019E577
:100C0C0042A2E713F8E555F4240138400B20E7081D
:100C1C007554FFF42401F555815AE8FAD3E813FC16
:100C2C008852C3EF94036020EF20E007E82CF8EC27
:100C3C00FA8146E8282402F87AFEC3EF94034008B0
:100C4C008A54884E8C50815A88548A4E8C50E56B4D
:100C5C00C3335002646BF56B3060028164753402EF
:0F0C6C00D26043E680E52D54066026A840A941DA
:100C7B00C3E913F9E813F8C2AF53E67F759100C3CC
:100C8B00E498F594E499F595759104D26043E68068
:100C9B00D2AF22D265754400752000306B037520EE
:100CAB0040020CBDD265754400752040306B037556
:100CBB002000D2AF7801206722E52D54066002C2D6
:100CCB0065C3E54194054013780294054008780309
:100CDB00940540027806306902780A206019E544D1
:100CEB00601530690AC3E53394034003D53406D24B
:100CFB00AFD26CA18E916CD2AF0000C2AF20672631
:100D0B00E541C3FB940F40027B0FEB2405307301CD
:100D1B0023306A02742820620123F9306902798238
:100D2B00E58BC39940B50544E59B5440B52002A122
:100D3B007830690A08C3E8940A40010881E6206507
:100D4B000281BDC26553E67F7591003067107594C3
:100D5B00007595FE759104D26043E68081BDAE406F
:100D6B00AF41C3E49EF594E49FF595A15FC3E533D2
:100D7B009402500281BD30650281BDD802A18C81E5
:100D8B00E6C26C53E67F7591008554948555957535
:100D9B009104854E56854F57D26043E680D2AFE51E
:100DAB002D54066008206A020533020DC8306C0D05
:100DBB00206B0A2065071581158102161D2278000C
:100DCB003064053065027801E53775F007A4F9E565
:100DDB00F028F5F0E9A2F013A2F113A2F213F53704
:100DEB00C394785003753778C3E53795384008D2EC
:100DFB0066D295D293D297306002C1028550568548
:100E0B005157D26043E68022207D11C2AF75430259
:100E1B00C296D294D2AF759F11020FE2C2AF754347
:100E2B0002C296D292D2AF759F11020FE23072437B
:100E3B00207D20C2AF754303900143757E40D29352
:100E4B00C292306204C297C156D296D2AF759F132D
:100E5B00020FE2C2AF754303900143757E40D295FA
:100E6B00C294306204C297C176D296D2AF759F10EE
:100E7B00020FE2207D17C2AF75430390011ED29380
:100E8B00306202C297D2AF759F13020FE2C2AF75E9
:100E9B00430390011ED295306202C297D2AF759F69
:100EAB0010020FE2207D11C2AF754304C294D2929F
:100EBB00D2AF759F10020FE2C2AF754304C292D23C
:100ECB0094D2AF759F13020FE2307243207D20C284
:100EDB00AF754305900132757E10D297C296306282
:100EEB0004C295C1F2D294D2AF759F11020FE2C228
:100EFB00AF754305900154757E04D297C29630624C
:100F0B0004C293E112D292D2AF759F11020FE2206D
:100F1B007D17C2AF754305900114D297306202C2A0
:100F2B0095D2AF759F11020FE2C2AF7543059001C9
:100F3B0028D2973062EBC293D2AF759F11020FE2AA
:100F4B00207D11C2AF754306C292D296D2AF759F68
:100F5B0013020FE2C2AF754306C294D296D2AF759D
:100F6B009F10020FE2307242207D20C2AF75430109
:100F7B00900154757E04D295C294306204C293E101
:100F8B008ED292D2AF759F10020FE2C2AF754301A2
:100F9B00900132757E10D293C292306204C295E1F9
:100FAB00AED294D2AF759F13E1E2207D16C2AF751E
:100FBB004301900128D295306202C293D2AF759F44
:100FCB0010E1E2C2AF754301900114D2933062027B
:100FDB00C295D2AF759F13C26622900112757E0027
:100FEB00D295D293D297C294C292C296C262227801
:100FFB008076070876070876010876040876FF08DE
:10100B0076FF08760A087602087601087601788C56
:10101B0076010876000876B40876FF0876FF087626
:10102B00FF0876030876FF0876010876FF08762519
:10103B000876D00876780876C80876040876FF0814
:10104B00760108760008767A08760A087601087623
:10105B00010876000876FF227887E6FFC272BF038D
:0F106B0002D2727888C27DE630E102D27DC27E69
:10107A007889E630E102D27EC3EF94026008758E69
:10108A0001D273021095758E00C273227880E6141D
:10109A009000809378A4F67881E614900080937883
:1010AA00A5F67886E61490008D9378A6F6789FE6E2
:1010BA00F8700108C3E8941140027811E82828F56D
:1010CA006E256E256E28F56F256E2828F570789C9A
:1010DA00E67538FF75390CB402067538A075390AF9
:1010EA00B4030675388275390578A3E61490009A18
:1010FA0093F569120FE522227896E6FA7897E6FBCD
:10110A007888E6B40305C3EB940EFB307F047A00BB
:10111A007BFFC3EB9AFCC3948250027C82757500F4
:10112A000575EC8575F0A4C3E5F0947D40F222D2F2
:10113A007F31021205687A007B007C1012055EE599
:10114A005F2AFA74003BFBDCF37C04C3EB13FBEA73
:10115A0013FADCF7FEC27F310222E5EF20E60375BF
:10116A0020000520903FFFE520146006901DFF1423
:10117A0060009304600375EF1253D9BF7581C043B1
:10118A00FF8012055975EF0243B203E5B324042028
:10119A00E70DF521E5E320E0068521B343E30112DB
:1011AA000FE57580FF75A40075F1B275D4DF7590EF
:1011BA00A975A5FC75F2FE75D50175A60175E24102
:1011CA00E4F8F6D8FD756B01120FFA1216657898D5
:1011DA008676753001C2AF12057212058212056851
:1011EA0012058912056812059012056812178812ED
:1011FA00057212057212056DC2AF78FA79FA308556
:10120A0007D9FBD8F7021C0011631196310131028C
:10121A0078988676120FE575885075891275C824F4
:10122A0075910475D84075A82275B80275E690754F
:10123A009B80759D0075D10E75BC5875BB0875BA33
:10124A001175E880120559D2AF1208B253DACF20CD
:10125A007E0343DA20307E0343DA1043DA01C2D830
:10126A00C271120572D2617B037A0CE55E70077A4D
:10127A000CDB03021202120568207003021202C27A
:10128A0070E55FC3940240E1E52F541F856160F564
:10129A0061B560D5DAD5C26153DACF207E0343DA6D
:1012AA0020307E0343DA10C2D8C27178A2E67008F1
:1012BA00D274E52F54E0F52FC27575290012056D19
:1012CA00307409C3E529940A4002D27512055E7882
:1012DA00023074027800C3E55F9840F0C2AF12058D
:1012EA0082120582120582D2AF120572754D001262
:1012FA00055E788CE6C3940150030213CFE530C330
:10130A00940150030213CF207435C3E55F94FF5054
:10131A00030213CFC2AF120597D2AF12056DC3E510
:10132A005F940150EFC2AF12058212056312058263
:10133A00D2AF12056DC3E55F94FF40E902180D7F35
:10134A0005D27F310212056DC2AFC27F3102AE5F94
:10135A00C3E55F947FD2AF4076120559C2AF12053A
:10136A0097D2AFDFDC3139C3EE94057897F61205D0
:10137A00721216A71217907F0AD27F310212056DD8
:10138A00C2AFC27F3102AE5FC3E55F947FD2AF5076
:10139A00E6120559C2AF120582120563120582D2FE
:1013AA00AFDFD63139EE24057896F6120572121699
:1013BA00A71217BF12056D3102C3E55F94FF5002F1
:1013CA00611102180DC3E55F954D4003855F4D120B
:1013DA00056D78017988E7B403027805C3E55F985B
:1013EA00400241F9C2AF120597120597120597D22A
:1013FA00AF120572753000E4F531F5320531E53189
:10140A00F470390532789AE6781914601278321431
:10141A00600D787D14600878FA146003753200C391
:10142A00E53298401715327531B478998676C2AF8D
:10143A00120597D2AF7898867612056D120563E584
:10144A002A7005307402410278012074027806C3BA
:10145A00E55F9840A712056DE52A7003021202C2E1
:0F146A00AF120FE5E4F522F523F524F525F5265D
:10147900F56AD2AF7885E6C333F568E4F545F546F4
:10148900F547F548F549F573F52CF52DF5377573DD
:101499000875BB10120559120945E5E820ECFBA8AF
:1014A900BDA9BEE97001F8887412094975730875F8
:1014B900BB107887E6FE760211637887EEF6C2AF35
:1014C9007564FF120A04852264852265852266D225
:1014D900AF75220175240175250175260185636C97
:1014E900756D017888E6B40307C27D307602D27D36
:1014F900D268D269753300120F4B120F70120A2489
:10150900120A2B120A24120A2B120A24021524C2C7
:10151900AF1163D2AF75730075BB08120CAF120619
:1015290062120DC9120E13120A2B120C9E306D0392
:1015390012070220670312085530670312089C122C
:101549000DC9120E38120A2B120CAF306D03120797
:101559003E120DC9120EAF120A2B120C9E306D03EA
:1015690012079C120DC9120ED4120A2B120CAF309D
:101579006D031207F9120DC9120F4B120A2B12092A
:1015890045120C9E120DC9120F70120949120A2B2D
:1015990030692F206B2C85676485676585636C7559
:1015A9006D0179187A0CC3E533994009C269D26A89
:1015B9008A350215CBC3E55F940140030215240265
:1015C9001625306A1B206B18E535147004C26AA110
:1015D90018F535C3E55F9401400302152402162569
:1015E900753600C3E5629401400985676585636CBA
:1015F900756D01C3E56278FA985021307404E52AC3
:10160900601A78F0306B058567647820C3E54198E6
:101619005002A1240536E55F6002C128753600C273
:10162900AF120FE57887E6FE760211637887EEF64A
:10163900E4F522F523F524F525F526F568C268D2E7
:10164900AF120559120FE5307406E52A70024102FE
:10165900788DE6C39401400241D68101901A0D7834
:10166900201216E9E520B4A50CA31216E9E520B469
:101679005A03021687120FFA1216A70216A6901A13
:101689000378807B0A1216E9A308DBF9901A0F7810
:101699008C7B181216E9A308DBF9901A2722C2AF2E
:1016A900121728121702901A00740E1216EEA3745C
:1016B900041216EEA374141216EE901A0378807BA6
:1016C9000A1216EDA308DBF9901A0F788C7B181211
:1016D90016EDA308DBF912173B121719901A2722E6
:1016E900E493F622E6438F01538FFD75EF0275B738
:1016F900A575B7F1F0538FFE22438F02438F017511
:10170900EF0275B7A575B7F1901A0DF0538FFC224A
:10171900901A0D74A5D1EE901A0E745AD1EE227A50
:101729003079D07820901A40D1E9E520F709A3DA79
:10173900F7227A3079D0901A40E7D1EE09A3DAF985
:1017490022AB77A878BB01027980BB02027981BB01
:1017590003027982BB04027994BB05027983BB0633
:10176900027986BB07027992BB08027987BB090215
:10177900799CBB0A027988BB0B027989E8F7227C3C
:1017890005120572DCFB22C2AF120582120589120D
:101799000590120597120563120582120589120533
:1017A9009012059712056312058212058912059098
:1017B900120597D2AF22C2AF1205971205901205F2
:1017C900891205821205631205971205901205897F
:1017D90012058212056312059712059012058912E6
:1017E9000582D2AF22AE77AF78C2AF120582120559
:1017F90082120582120563DEF2120597120563DF74
:10180900F8D2AF221217901217881217887577012C
:101819007578017579001217EE7C05AD5F120572B6
:10182900C3ED955F70F5C3E55F9401400AC3E55FB9
:1018390094FF403702185112174A1216A71217902F
:10184900C2AF75EF12121788DCD10579C3E5799417
:1018590003500280C11217880578E5771490009F1C
:0E18690093F808C3E57898500280A8121788FB
:101877001217880577C3E577940C50028094120FEE
:0C188700FA1216A7C2AF75EF12121788F4
:0319FD0002116470
:101A00000E041407070104FFFF0A020101A55A0191
:101A100000B4FFFFFF03FF01FF25D078C804FF01DA
:081A200000FF0A010100FFFFB5
:101A4000235475726E6967794E6665743138412327
:101A500023424C48454C4923463333302320202031
:101A60002020202020202020202020202020202076
:101C0000C2AFC2D353D9BF7581C043B20343FF8073
:101C1000752438752503B1C975EF0275E24043F1AB
:101C20002053A4DF75D400D2857DFA780379E67C51
:101C300010752200752300901DD67B0675249875BB
:101C400025013085028142208508D8FBD9F9DCF7CF
:101C500081B4308508D8FBD9F9DCF781B4B189E4C7
:101C600093A3C39A6004DDC381B4DBDBB17B600264
:101C7000812B7B08E493FAA3B15CDBF87A30B15C8A
:101C8000752200752300B17BEAFCEBFDC3ED94FEE9
:101C9000400EB17B8A278B28ED30E0048A828B834B
:101CA000B17B7AC270D8C3ED94FE601350CEBD00F4
:101CB00025EC60097520007521FF0200008100A855
:101CC00027A9280809D804D90281D3B17FEA89AAB3
:101CD000F281C50D81A0C3ED94035049EDA2E092BD
:101CE000007AC5C3E5829400E583941C50902000DF
:101CF00010438F02438F0175B7A575B7F1F030001F
:101D00001FA827A9280809438F01538FFDD804D99C
:101D100002A12089AAE275B7A575B7F1F0A3A10DBC
:101D2000538FFC817C7AC1BD030CE493A3FAB140CC
:101D3000DCF8B138817C817EAA22AB23B15CEBFA5E
:101D4000EA6222752608C3E52313F523E52213F57D
:101D50002250066323A0632201D526EAB1C9B1C986
:101D600075260AEAF4200102D285300102C285B14B
:101D7000C9C3134002C201D526EB22B17FEAFB2082
:101D80008502A17F308502A184752608AE24AF2587
:101D9000C3EF13FFEE13FEB1CDB1C9C3EA13308513
:101DA000024480FA30E703632201C3E52313F523DD
:101DB000E52213F52250066323A0632201D526D91C
:101DC000E52265236523F52222AE24AF250E0FDE22
:101DD000FEDFFCD20122424C48656C693437316326
:041DE000F3300601D5
:00000001FF
